:100000000C941E060C94D3270C9400280C944606DE
:100010000C9446060C9446060C9446060C94460630
:100020000C9446060C9446060C94EF120C9446066B
:100030000C9446060C9446060C9446060C94460610
:100040000C942D280C9446060C941B2C0C945E2CBE
:100050000C9446060C9446060C9446060C944606F0
:100060000C9446060C9446065318B5189418971825
:100070009A189D18A018A318A618B518AF18E71954
:10008000E919E919E719E919E919E919E919E91962
:10009000E919E919E919E919E919E919E919E91950
:1000A0006D19E919E919E919E919E919DE18E919C8
:1000B000E919E919E919E919E919E919E919E91930
:1000C000E919E919E919E919E919E9197919791900
:1000D0007919791979197919791979197919E91920
:1000E000E919E919E919E919E919DE1878197819EE
:1000F00078197819E91986198C19921998199E1985
:10010000A419AA19B019BA19C419CE19D8191F19E6
:10011000E118E919E919E919E9196D19E919E91954
:10012000E919E919E919E919E919E91977197719A3
:1001300077197719E91986198C19921998199E1946
:10014000A419AA19B019BA19C419CE19D8191F19A6
:10015000E118E919E919E919E9196D191C1A1C1AAC
:100160001C1A1C1A1C1A1C1A1C1A1C1A1C1A1C1ADF
:100170001C1A1C1A1C1A331B331B331B331B331B57
:10018000331B611A6B1A751A7F1ADD1AE71AF61AF1
:10019000071B8F1CA41CB01CB91CC81CED1CF61C32
:1001A0003F1D081D522058205E2065207320952099
:1001B000B320456E746572206D656E752E2E2E000F
:1001C000546F67676C6564206D6963726F50504D42
:1001D00000546F67676C656420696E76657274653C
:1001E000642050504D2100546F67676C6564205443
:1001F00058206D7574696E672100546F67676C6570
:10020000642074656C656D65747279210050726F3D
:10021000746F636F6C206572726F72207769746897
:100220002052580054696D656F7574207768656E4B
:1002300020636F6E6E656374696E6720746F205201
:100240005800507265737320616E79206B65792058
:10025000746F2063616E63656C00436F6E6E6563DF
:1002600074696E6720746F2052582C20706F776508
:100270007220757020746865205258202877697440
:10028000682062696E6420706C7567206966206EF4
:100290006F74207573696E6720616C776179732064
:1002A00062696E642900546F67676C656420276912
:1002B0006D6D656469617465206F75747075742700
:1002C00000546F67676C65642027736C61766520E6
:1002D0006D6F64652700546F67676C6564202761E4
:1002E0006C776179732062696E642700546F676769
:1002F0006C65642050504D206368616E6E656C20A3
:100300006C696D69740053657420525353492069B8
:100310006E6A656374696F6E206368616E6E656C8A
:100320002028303D3D64697361626C652900536526
:10033000742050504D206D696E696D756D20737914
:100340006E630053657420626561636F6E20696E31
:1003500074657276616C0053657420626561636FC9
:100360006E2064656C617900536574206265616319
:100370006F6E206672657175656E637920696E2097
:10038000487A3A20303D64697361626C652C205074
:10039000783D504D52206368616E6E656C20782CFC
:1003A0002046783D465253206368616E6E656C202E
:1003B00078005365742050574D2073746F7020641B
:1003C000656C61792028302064697361626C6564B2
:1003D0002C20312D323535203D3D20302E317320FB
:1003E0002D2035306D696E29005365742050504DB5
:1003F0002073746F702064656C61792028302064EC
:10040000697361626C65642C20312D323535203D75
:100410003D20302E3173202D2035306D696E29003E
:10042000536574206661696C736166652064656CF0
:1004300061792028302064697361626C65642C20C6
:10044000312D323535203D3D20302E3173202D2089
:1004500035306D696E29002A2A2A2A2A2A2A2A2A50
:100460002A2A2A2A2A2A2A2A2A2A2A2A2A2A2A2AEC
:100470002A2A2A2A0052582041636B6564202D20C5
:1004800072657665727420737563636573736675E0
:100490006C21002A2A2A2A2A2A2A2A2A2A2A2A2AAD
:1004A0002A2A2A2A2A2A2A2A2A2A2A2A2A2A2A2AAC
:1004B000002A2A2A2A2A2A2A2A2A2A2A2A2A2A2AC6
:1004C0002A2A2A2A2A2A2A2A2A2A2A2A2A2A00528E
:1004D000582041636B6564202D20757064617465DC
:1004E000207375636365737366756C21002A2A2A0D
:1004F0002A2A2A2A2A2A2A2A2A2A2A2A2A2A2A2A5C
:100500002A2A2A2A2A2A2A2A2A2A0056616C696457
:100510002063686F69636573206172653A205B319F
:100520005D2D5B31365D20286368616E6E656C20E1
:10053000312D31362900536574206F7574707574D0
:1005400020666F7220706F727420005B585D2061AE
:10055000626F7274206368616E67657320616E6498
:10056000206578697420525820636F6E6669670051
:100570005B535D20736176652073657474696E6783
:100580007320746F205258005B525D20726576654F
:1005900072742052582073657474696E6773207486
:1005A0006F2064656661756C747300557365206EA9
:1005B000756D62657273205B312D445D20746F2010
:1005C0006564697420706F727473205B452D515D92
:1005D00020666F722073657474696E677300202DD6
:1005E00020726563656976657220636F6E66696700
:1005F000757261746F722C20727820737720000AF4
:100600000A6F70656E4C52536E67200053657420FC
:1006100073657269616C2062617564726174653AB8
:10062000200056616C69642063686F696365733A82
:100630002031202D20342B34202F2032202D203823
:10064000202F2033202D20382B34202F2034202D14
:10065000203132202F2035202D2031322B34202FF5
:100660002036202D20313600536574204368616E9A
:100670006E656C20636F6E6669673A20005365741F
:100680002044617461726174652028302D32293AEA
:10069000200053657420486F70206368616E6E653A
:1006A0006C7320286D61782032342C207365706162
:1006B000726174656420627920636F6D6D61732966
:1006C0002076616C69642076616C75657320312DCC
:1006D0003235353A2000536574206368616E6E656B
:1006E0006C2073706163696E6720287831306B48C5
:1006F0007A293A200053657420524620706F77653E
:10070000722028302D37293A200053657420524634
:10071000206D6167696320286865782920652E67E8
:100720002E20307844454144463030443A2000532E
:1007300065742062617365206672657175656E63AC
:10074000792028696E20487A293A20005B5A5D207A
:10075000656E746572207265636569766572206383
:100760006F6E66696775726174696F6E2075746902
:100770006C79005B465D20646973706C61792061FF
:10078000637475616C206672657175656E63696509
:10079000732075736564005B525D2063616C6375E3
:1007A0006C6174652072616E646F6D206B65792079
:1007B000616E6420686F70206C697374005B495DC2
:1007C000207265696E697469616C697A6520736508
:1007D0007474696E677320746F20736B65746368DB
:1007E0002064656661756C7473005B585D2072658A
:1007F00076657274206368616E67657320616E64EC
:100800002065786974206D656E75005B535D20739B
:100810006176652073657474696E677320746F20E8
:10082000454550524F4D20616E64206578697420B3
:100830006D656E7500557365206E756D62657273BA
:10084000205B302D395D20746F20656469742070E1
:100850006172616D657465727300202D2053797328
:1008600074656D20636F6E66696775726174696F18
:100870006E000A0A6F70656E4C52536E672000510D
:1008800029204F7574707574206265666F726520DB
:100890006C696E6B20283D465329203A2000502970
:1008A00020536C617665206D6F64652028657870D3
:1008B0006572696D656E74616C293A20004F29205C
:1008C00054696D65642042494E44206174207374FC
:1008D000617274757020203A20004E292050504DCE
:1008E000206F7574707574206C696D69746564200F
:1008F000202020203A200044495341424C454400E6
:100900004D292050504D205253534920746F20637D
:1009100068616E6E656C202020203A20004C2920F2
:1009200050504D206D696E696D756D2073796E63E1
:10093000202875732920203A200044495341424C15
:100940004544004B29204661696C736166652062ED
:100950006561636F6E20696E74762E2028312D32AA
:10096000353573293A20004A29204661696C736144
:10097000666520626561636F6E2064656C617920D5
:1009800028302D323535203D3E20313073202D204A
:100990003135306D696E293A200049292046616958
:1009A0006C7361666520626561636F6E206672714B
:1009B0002E203A200048292050574D2073746F7024
:1009C0002064656C6179202020202020203A2000BE
:1009D00047292050504D2073746F702064656C61FE
:1009E00079202020202020203A200046292046611E
:1009F000696C736166652064656C617920202020D4
:100A00002020203A200050574D206368616E6E65AB
:100A10006C200066756E6374696F6E3A2000292041
:100A2000706F72742000506F776572546F776572C3
:100A300000445446205548462033322D62697420C4
:100A400031306368004F70656E4C52536E67525878
:100A5000206D696E6920342F36636800466C7974A6
:100A6000726F6E2F4F72616E6765525820554846FF
:100A70002038636800525820747970653A20004429
:100A8000697361626C656400487A00203D3D200016
:100A900043616C63756C61746564207061636B6540
:100AA0007420696E74657276616C3A200042292068
:100AB0004D6963726F202868616C66292050504D23
:100AC000202020203A00412920496E766572746505
:100AD000642050504D20696E20202020203A0030A4
:100AE00029204D7574652062757A7A657220286DAB
:100AF0006F73746C79293A003929205365726961E2
:100B00006C2062617564726174653A00736D617224
:100B100074506F7274004672536B79005472616E38
:100B200073706172656E740044697361626C6564B0
:100B30000038292054656C656D657472793A2020FF
:100B40002020202020003729204368616E6E656CCC
:100B500020636F6E6669673A202000362920446161
:100B60007461726174652028302D32293A2020206A
:100B700000352920486F70206368616E6E656C7364
:100B80003A2020202020003429204368616E6E65C1
:100B90006C2073706163696E673A202000332920EE
:100BA000524620706F7765722028302D37293A2001
:100BB0002020003229205246206D616769633A2067
:100BC0002020202020202020003129204261736530
:100BD000206672657175656E63793A202020000089
:100BE00000000700020100000304060000000000EE
:100BF00000000001020408102040800102040810D7
:100C00002001020408102004040404040404040263
:100C10000202020202030303030303000000002395
:100C2000002600290000000000250028002B0000FD
:100C3000000000240027002A00004C2D11241FBEB4
:100C4000CFEFD8E0DEBFCDBF13E0A0E0B1E0E6EA31
:100C5000F0E602C005900D92A83CB107D9F716E066
:100C6000A8ECB3E001C01D92AE38B107E1F71CE07B
:100C7000CCE3DCE004C02297FE010E94552ECA336B
:100C8000D107C9F70E94882D0C9451300C940000B4
:100C900080917305813019F482E08093730580910F
:100CA0007305833019F484E0809373050895A89543
:100CB0000895DC01ED91FC910190F081E02D099502
:100CC00008952091740530917505382748E0C901D1
:100CD000880F991F37FF06C09C0151E2252750E17C
:100CE000352701C09C01415091F730937505209341
:100CF0007405089588E38093760580E092ECA1E086
:100D0000B0E08093770590937805A0937905B09330
:100D10007A0587E08093830580EC9AECA9E8B6E336
:100D200080937B0590937C05A0937D05B0937E0511
:100D300085E0809384058DEE9EEFADEABEED809355
:100D40007F0590938005A0938105B0938205E5E827
:100D5000F5E080E090E0863028F4DC01AE54BC4F32
:100D60002C9101C020E0219301968831910599F7DB
:100D700082E080939D058AE080939E05089580EC33
:100D800097EFAAEBB7E38093BB059093BC05A093C4
:100D9000BD05B093BE0580E090E0A0E0B0E5809393
:100DA000BF059093C005A093C105B093C205E3ECC5
:100DB000F5E080E081938F5F8031E1F70895A0E056
:100DC000B0E0E5EEF6E00C941E2ED82F0E948328AA
:100DD0006115710581059105C9F30E94C12E10921C
:100DE0007F05109280051092810510928205C4E063
:100DF000812C912C54018A94C0907F05D09080055D
:100E0000E0908105F0908205FE2CED2CDC2CCC24AA
:100E10000E94BC2EA50194010E94FD2D6C0D7D1D2C
:100E20008E1D9F1D60937F057093800580938105C3
:100E300090938205C15001F7DD2309F450C005E805
:100E400015E0E801A12CB12C62E3C62ED12CE12CD7
:100E5000F12C8881882309F442C0B39419F40E94CC
:100E60007A063DC00E94BC2EA70196010E94FD2D6E
:100E7000E1E0E60FA5E8B5E08A2F801B8A1520F493
:100E80008D918E13F9CFE9CF2091840530E0A0E158
:100E9000B7E20E94952D9B01AC01AE2FB0E00E94FD
:100EA000A42D40907B0550907C0560907D0570904E
:100EB0007E05640D751D861D971D4090BB055090E5
:100EC000BC056090BD057090BE05461657066806C5
:100ED000790618F2E993A39488E1A812BACFCDB7A6
:100EE000DEB7E0E10C943A2E8436910520F4BC0183
:100EF00080E090E017C09C018E3B910528F42A55B4
:100F00003109AAE0B0E00CC0823D910528F4245BD1
:100F10003109A4E6B0E004C02D5C3109A8E5B2E0D7
:100F20000E94952DA4E6B0E09B01AC010E94A42D87
:100F3000089590E08C599F4F0E947407089561E0D6
:100F40008FE00E94302960E08FE00E9469290895B7
:100F5000892B11F061E001C060E08FE00E946929F7
:100F6000089560E08CE00E94302961E08BE00E94EF
:100F7000302961E08DE00E94302960E082E00E942B
:100F8000302961E084E00E943029089542E050E079
:100F900068E476E080E00E94B3270895E3E0F0E0A3
:100FA00089E080935700E491E67081E0E63009F033
:100FB00080E00895CF93DF93C82F0E94CE07882347
:100FC00081F0DFB781E080937205F8940E945706A4
:100FD00088E180936000C0936000C1110E945706B1
:100FE000DFBFDF91CF9108958F929F92AF92BF9212
:100FF000CF92DF92EF92FF92CF93FC01C0A5EC2F2E
:10100000E770F0E0E658FC4FA081B0E0C7FF03C0F6
:1010100024E130E002C02FE030E0FC0197A183E141
:10102000989FF0011124E25CFE4F80809180A280A5
:10103000B380A20FB31F20E43FE14DE750E00E94D0
:10104000AF2DA50194010E94DB2D8C2F887149F4EE
:1010500069017A01E0EDCE0EE7E0DE1EE11CF11C35
:101060001BC0C7FF05C060E47AE88CE29EE004C0C4
:1010700060E07EEE8AEB9BE069017A01F8EBCF0E2F
:10108000FBE0DF1EE11CF11CA50194010E94DB2D99
:10109000C20ED31EE41EF51EC701B60169517C4F76
:1010A0008F4F9F4F28EE33E040E050E00E94DB2D51
:1010B000A8EEB3E00E94A42DCF91FF90EF90DF90B7
:1010C000CF90BF90AF909F908F9008958F3F9105E4
:1010D00051F048F0811522E0920738F081159340D5
:1010E00030F482E0089580E0089581E0089583E07F
:1010F0000895A0E0B0E0EFE7F8E00C94272EEB01B4
:101100008A01B82FB695A0E028813981F8012083A3
:101110002A813B8121832C813D8122832E813F8145
:101120002383688179814A815B812C813D81EE81B5
:10113000FF819F2F9295990F990F907C272F2370F5
:10114000922B252F2370220F220F922B232F2370F7
:101150002295207F922BF80194830B5F1F4F2896D6
:10116000AF5FBA1788F680FF24C0888199810E94FA
:101170006608D82E8A819B810E946608E82E8C81A1
:101180009D810E946608F82E8E819F810E946608CC
:10119000F0E4DF9EA001112490E1E99E900111246A
:1011A000242B282BE4E0FE9EB0011124262BF8010D
:1011B0002083CDB7DEB7E7E00C94432E803223E0E6
:1011C000920708F1883E23E0920740F48F51934044
:1011D000E4E096958795EA95E1F70895803D27E04C
:1011E000920718F48C5D93400895883928E092079F
:1011F00068F4885C974074E0969587957A95E1F756
:101200008D509C4F089580E090E008958FEF93E01B
:1012100008958C30910540F4A4E0880F991FAA9599
:10122000E1F7885D9C4F0895843F23E0920718F40E
:1012300084529C4F0895811524E0920740F486570C
:10124000934FF4E0880F991FFA95E1F7089580E92C
:1012500098E008959C013695279525753575821B74
:10126000930B9C0123733373969587959695879579
:1012700083739373820F931F9C0154E036952795D7
:101280005A95E1F7280F391F2F703F7041E051E068
:10129000249FC001259F900D349F900D1124892F0C
:1012A00008952D98882319F000002B9A02C00000A1
:1012B0002B9800002D9A000008952D9A000083B10C
:1012C0002D980000829581700895CF93DF93D82FD9
:1012D0005C9A2D985C98C8E08D2F80780E94510907
:1012E000DD0FC150C9F72D98DF91CF9108958F7709
:1012F0000E9465090895CF93DF93D82FC8E08D2F02
:1013000080780E945109DD0FC150C9F72D98DF91F7
:10131000CF910895CF93DF932D98C8E080E0D82F28
:10132000DD0F0E945D098D0FC150C9F7DF91CF918C
:1013300008950E9477090E948A095C9A0895A1E0A5
:10134000B0E0E5EAF9E00C942C2E806869830E94F5
:1013500065096981862F0E947B095C9A2196E2E0EB
:101360000C94482ECF93C0917F05C827E82FF0E05A
:10137000EA58FA4F678589E70E949F096C2F8DE331
:101380000E949F096C2F82E40E949F09CF910895CB
:1013900086E20E9499090895CF93DF93EC016C8156
:1013A0008CE10E949F096D818DE10E949F096E81F1
:1013B0008EE10E949F096F8180E20E949F096885EB
:1013C00081E20E949F09698582E20E949F096A85E5
:1013D00083E20E949F096B8584E20E949F096C85CD
:1013E00085E20E949F096D858AE20E949F096E85B1
:1013F0008EE60E949F096F858FE60E949F0968898B
:1014000080E70E949F09698981E70E949F096A8994
:1014100082E70E949F09DF91CF910895CF92DF92DA
:10142000EF92FF92CF93DF936B017C01C11488E3AD
:10143000D8068CE9E8068CE1F80628F5C701B60164
:1014400020E836E948E950E00E94DB2DE901689781
:1014500060E879E687E69FEF0E94B72D6C0D7D1D51
:101460008E1D9F1DF2E0660F771F881F991FFA954A
:10147000D1F721E732E040E050E00E94DB2DF22E70
:10148000E32E80E421C0C701B60120E03DE241E344
:1014900051E00E94DB2DE901689760E073ED8EEC6E
:1014A0009EEF0E94B72D6C0D7D1D8E1D9F1D660F3A
:1014B000771F881F991F21E732E040E050E00E942B
:1014C000DB2DF22EE32E80E66C2F6F71680F85E71F
:1014D0000E949F096E2D86E70E949F096F2D87E766
:1014E0000E949F09DF91CF91FF90EF90DF90CF9006
:1014F0000895682F8DE60E949F0908958F929F920C
:10150000AF92BF92CF92DF92EF92FF92CF93DF9391
:10151000D82F83E00E9499098093710584E00E948E
:1015200099098093700560E086E00E949F0961E060
:1015300087E00E949F096FE789E00E949F0965E0AC
:101540008AE00E949F0962E18BE00E949F0965E1A9
:101550008CE00E949F096DEF8DE00E949F0960E082
:101560008EE00E949F09DD2319F08BE291E008C014
:1015700020919D0533E1239FC0011124825C9E4F81
:101580000E94CC096CE880E30E949F096FE082E32F
:101590000E949F0962E483E30E949F0980919E0557
:1015A00087FF02C064E101C06AE084E30E949F09F2
:1015B0006AE285E30E949F096DE286E30E949F092B
:1015C00064ED87E30E949F0960E088E30E949F0921
:1015D00060E089E30E949F09D11109C0C0907F0596
:1015E000D0908005E0908105F090820507C0C5E9A4
:1015F000CC2EC1ECDC2EED2CCEEDFC2ECAE38F2CD4
:101600009924AA24BB24682D8C2F0E949F09682D41
:1016100085E08C0F0E949F09FE2CED2CDC2CCC2445
:10162000CF5FCE3361F76FEF83E40E949F096FEFC6
:1016300084E40E949F096FEF85E40E949F096FEF89
:1016400086E40E949F09DD2311F066E002C06091EC
:1016500083058DE60E949F0960E089E70E949F094B
:10166000609184058AE70E949F0960E083E70E94F9
:101670009F0960E084E70E949F09D11109C0609131
:101680007B0570917C0580917D0590917E0504C05D
:1016900060EC7AEC89E896E30E940E0ADF91CF9124
:1016A000FF90EF90DF90CF90BF90AF909F908F9082
:1016B000089561E087E00E949F0964E28EE70E943E
:1016C0009F0963E088E00E949F0960E088E00E9433
:1016D0009F0965E087E00E949F0962E085E00E9423
:1016E0009F0983E00E9499098093710584E00E941C
:1016F000990980937005089583E00E949909809369
:10170000710584E00E9499098093700561E087E08B
:101710000E949F096AE070E080E090E00E94A628A5
:101720000E94590B00000895CF92DF92FF920F9311
:101730001F93CF93DF931F92CDB7DEB7082F162FDD
:101740008EE399830E949F09F02EC02E9981D92E95
:101750008C2D8F19811738F4F60161916F018FE795
:101760000E949F09F5CF64E085E00E949F0983E015
:101770000E9499098093710584E00E9499098093E1
:1017800070050E94832860936C0570936D058093AB
:101790006E0590936F0569E087E00E949F0981E0E4
:1017A000809373050F90DF91CF911F910F91FF9060
:1017B000DF90CF9008950F931F930E94940B809118
:1017C0007305813099F40E94832800916C05109173
:1017D0006D0520916E0530916F05601B710B820BBA
:1017E000930B603A76488140910548F380917305E8
:1017F000813031F46EE971E082EE95E00E946F2A4B
:101800001F910F9108950F931F938091730582305C
:1018100021F41092730581E020C08091730581301E
:10182000D9F40E94832800916C0510916D052091D8
:101830006E0530916F05601B710B820B930B613A43
:1018400076488140910540F061E087E00E949F0961
:101850001092730582E001C080E01F910F910895FE
:10186000CF93DF93EC014AE050E06D2F70E082EE01
:1018700095E00E943D2B6EE282EE95E00E94412AA7
:10188000BE0184E0769567958A95E1F76F707727BA
:101890004AE050E082EE95E00E943D2B6EE282EE3F
:1018A00095E00E94412ABE016F7077274AE050E020
:1018B00082EE95E00E943D2BDF91CF910895D82FC5
:1018C000C0E0CD1790F45E9A409A64E670E080E044
:1018D00090E00E94A6285E98409864E670E080E060
:1018E00090E00E94A628CF5FECCF6CE271E080E030
:1018F00090E00E94A628E4CF0F931F93CF93DF932D
:10190000EC01062F15E0115051F0CE010E94383045
:10191000081741F0602FCE010E944030F4CF82E0E2
:101920000E945F0CDF91CF911F910F910895A0E06D
:10193000B0E0EDE9FCE00C941E2E482E562EC0E0DF
:10194000D0E0612C712CE12CF12C00E010E0411072
:101950000CC06090D40586E4689E3001112459E1E2
:10196000E52EF12C0AEB15E01EC091E049120FC0E4
:101970006090D405E6E46E9E30011124FBE16F0E09
:10198000711C49E2E42EF12C06E715E00CC082E060
:10199000481209C028E1622E77247394EE24E39460
:1019A000F12C03ED15E043018C0E9D1E1092750580
:1019B000109274053401A62CA818B12CC30101960D
:1019C0006C01AE14BF04A8F4A00EB11E511006C0E5
:1019D000C3010E943830F501808305C0F5016081A4
:1019E000C3010E947C0CF50180810E9461063601D2
:1019F000E2CFC301511018C0C3010E943830B82E85
:101A0000C6010E9438302B2D30E0322F2227282BA0
:101A100080917405909175058217930779F4C0E061
:101A2000D0E05524539493CF3601609175050E9400
:101A30007C0C60917405C6010E947C0CC05EDE4F78
:101A4000C13E92E0D90708F482CF852DCDB7DEB72D
:101A5000E0E10C943A2E61E082E00E94970C089538
:101A600060E082E00E94970C8091D305853020F0E1
:101A70001092D3050E942B0D8091D3058093D4053D
:101A8000089561E080E00E94970C61E081E00E948F
:101A9000970C089560E080E00E94970C882351F035
:101AA00060E081E00E94970C882321F08091760508
:101AB000883349F00E94BF060E947A0681E00E94A6
:101AC000DF060E94410D0895882319F06AEA71E04B
:101AD00002C06EEA71E082EE95E00E946F2A0895DE
:101AE000FF920F931F93CF93DF9369EC7BE082EE1D
:101AF00095E00E941B2A40917B0550917C056091E6
:101B00007D0570917E052AE030E082EE95E00E942E
:101B1000442B63EB7BE082EE95E00E941B2A409110
:101B20007F0550918005609181057091820520E1CB
:101B300030E082EE95E00E94442B6DE97BE082EE7E
:101B400095E00E941B2A4AE050E06091830582EEF6
:101B500095E00E946C2B67E87BE082EE95E00E94A6
:101B60001B2A4AE050E06091840582EE95E00E94D5
:101B70006C2B61E77BE082EE95E00E941B2AC5E8B2
:101B8000D5E0F12C8E0188818823A9F0FF2031F067
:101B900061EB71E082EE95E00E943E2A21964AE0D8
:101BA00050E0F801608182EE95E00E94352BF394BD
:101BB000F8E1FF12E7CF82EE95E00E94492A6BE53B
:101BC0007BE082EE95E00E941B2A4AE050E06091A3
:101BD0009D0582EE95E00E946C2B66E47BE082EE30
:101BE00095E00E941B2AE0919E05E770F0E0EE0F61
:101BF000FF1FEE57FC4F6081718182EE95E00E94DD
:101C00006F2A61E37BE082EE95E00E941B2A8091BF
:101C10009E058871883069F028F4811113C068E24C
:101C20007BE00CC0803141F0883161F46CE07BE0F6
:101C300005C06CE17BE002C066E17BE082EE95E0EE
:101C40000E945D2A68EF7AE082EE95E00E941B2AEE
:101C500040917705509178056091790570917A05EA
:101C60002AE030E082EE95E00E94442B6FED7AE0AE
:101C700082EE95E00E941B2A8091BF0580710E9430
:101C8000640D66EC7AE082EE95E00E941B2A80915A
:101C9000BF0580740E94640D6DEA7AE082EE95E0E3
:101CA0000E941B2A8091BF0580720E94640D60E92A
:101CB0007AE082EE95E00E941B2A86E795E00E947A
:101CC000F407AB01BC012AE030E082EE95E00E940F
:101CD000262B6BE87AE082EE95E00E941B2A86E7CD
:101CE00095E00E94F4079B01AC0160E472E48FE090
:101CF00090E00E94DB2DBA01A9012AE030E082EEDB
:101D000095E00E94262B68E87AE082EE95E00E943A
:101D10005D2ACDB7DEB7E5E00C94452E8F929F92F9
:101D2000AF92BF92CF92DF92EF92FF92811107C0E4
:101D30006FE77AE082EE95E00E945D2A2FC090E086
:101D40000E94740724E630E040E050E00E94DB2D62
:101D5000CA01B9012AE030E040E050E00E94DB2DEA
:101D600049015A016B017C012AE030E0B501A40170
:101D700082EE95E00E94262B6EE282EE95E00E94B4
:101D8000412A2AE030E0B701A60182EE95E00E94E8
:101D9000262B63E782EE95E00E94812AFF90EF9068
:101DA000DF90CF90BF90AF909F908F9008951F933A
:101DB000CF93DF9365E77AE082EE95E00E941B2ADD
:101DC00080919F05813041F46CE57AE082EE95E0E8
:101DD0000E945D2A10E050C0823019F465E47AE078
:101DE000F5CF843019F461E37AE0F0CF853091F7D4
:101DF00066E27AE0EBCFC12FD0E0C930D1050CF418
:101E000041C068E3610F82EE95E00E94412A6EE1D5
:101E10007AE082EE95E00E941B2ABE016F5F7F4F41
:101E20004AE050E082EE95E00E94052B63E17AE003
:101E300082EE95E00E941B2AC156DA4FE981E0321A
:101E400018F566E07AE082EE95E00E941B2A89810F
:101E5000803130F06DE673E082EE95E00E943E2A1C
:101E600069816F7070E06F5F7F4F4AE050E082EEF3
:101E700095E00E940E2B1F5F80914805181708F40B
:101E8000BACF0FC061E3BECFEF70F0E0EE0FFF1FDF
:101E9000EE56FC4F6081718182EE95E00E946F2AC0
:101EA000EACF6BEE79E082EE95E00E941B2A8091EA
:101EB000B7050E948E0E60ED79E082EE95E00E94FB
:101EC0001B2A8091B8050E948E0E65EB79E082EEA8
:101ED00095E00E941B2A8091B9050E948E0E6AE946
:101EE00079E082EE95E00E941B2A4091AF05509167
:101EF000B0056091B1057091B205411551056105BC
:101F0000710539F12AE030E082EE95E00E94442B21
:101F100067E679E082EE95E00E941B2A8091B30586
:101F20000E949907AB01BC012AE030E082EE95E007
:101F30000E94442B63E479E082EE95E00E941B2A24
:101F40004AE050E06091B40582EE95E00E946C2B6F
:101F500006C06AE379E082EE95E00E945D2A6DE1B9
:101F600079E082EE95E00E941B2A6091B5057091A0
:101F7000B6054AE050E082EE95E00E94562B60E004
:101F800079E082EE95E00E941B2A6091AE056034F4
:101F900050F470E06F5F7F4F4AE050E082EE95E0D2
:101FA0000E940E2B06C067EF78E082EE95E00E945B
:101FB0005D2A6AED78E082EE95E00E941B2A80910E
:101FC000AD0580FF03C063EB71E002C067EB71E019
:101FD00082EE95E00E946F2A6DEB78E082EE95E04C
:101FE0000E941B2A8091AD0582700E94640D6EE9EB
:101FF00078E082EE95E00E941B2A8091AD05847006
:102000000E94640D6FE778E082EE95E00E941B2A43
:102010008091AD0588700E94640DDF91CF911F9172
:1020200008950F931F93CF93DF93209145052F3F82
:10203000A9F56FEF75E082EE95E00E941B2A82E819
:1020400093E00E94300C6EED75E082EE95E00E9408
:102050001B2A80914605909147050E94300C6BEA3F
:1020600075E082EE95E00E945D2A68E875E082EEF8
:1020700095E00E945D2A60E775E082EE95E00E949F
:102080005D2A6BE475E082EE95E00E945D2A82EEA7
:1020900095E00E94492A0E94D70E68C012160CF0E3
:1020A00065C0332727FD30958091480590E0821761
:1020B00093070CF45BC066E375E082EE95E00E9446
:1020C0001B2A60914505772767FD70954AE050E02F
:1020D00082EE95E00E940E2B6BE075E082EE95E0BB
:1020E0000E941B2A10E008E2809149051817D0F5DC
:1020F000C12FD0E0CC0FDD1FC65BDA4F288130E066
:1021000080914505992787FD9095019728173907F4
:1021100039F56BEB71E082EE95E00E943E2A4AE0D1
:1021200050E0602F82EE95E00E94352B6FEB71E05E
:1021300082EE95E00E943E2AE981EF70F0E0EE0F1A
:10214000FF1FEE56FC4F6081718182EE95E00E9488
:102150003E2A63EC71E082EE95E00E943E2A0F5F1A
:102160001F5FC2CF82EE95E00E94492ADF91CF9196
:102170001F910F910895FF920F931F93CF93DF93B9
:10218000C5E8D5E0F12C8E0188818823D1F165EC7A
:1021900071E082EE95E00E943E2A4AE050E06F2D09
:1021A00082EE95E00E94352B62ED71E082EE95E0C3
:1021B0000E943E2A2196F801208130E0A0E1B7E29A
:1021C0000E94952D9B01AC01A0918405B0E00E9476
:1021D000A42DAB01BC0180917B0590917C05A09161
:1021E0007D05B0917E05480F591F6A1F7B1F2AE0AD
:1021F00030E082EE95E00E94442BF394F8E1FF1268
:10220000C2CFCDB7DEB7E5E00C94452E1092DF04C7
:1022100085E6E0EEF4E0DF011D928A95E9F7089586
:10222000CF93C82F8F3719F0883009F045C0E0915F
:10223000DF04EE23D9F1E150E093DF04F0E0E05257
:10224000FB4F10826DE070E082EE95E00E9459062F
:10225000C0E08091DF04C81760F4EC2FF0E0E0529A
:10226000FB4F608170E082EE95E00E945906CF5FDF
:10227000F0CF60E270E082EE95E00E9459066DE0DA
:1022800070E082EE95E00E945906C0E08091DF0484
:10229000C81778F5EC2FF0E0E052FB4F608170E05A
:1022A00082EE95E00E945906CF5FF0CF67E082EEA4
:1022B00095E00E94412A1DC08B3119F40E9406113D
:1022C0001AC08D30C1F08A30B1F08091DF048436BD
:1022D00068F76C2F70E082EE95E00E945906E0915D
:1022E000DF0481E08E0F8093DF04F0E0E052FB4FCB
:1022F000C08380E001C081E0CF910895CF93C82FC3
:102300000E9483286093C8047093C9048093CA0410
:102310009093CB04C093DD04CC2329F040E051EE30
:1023200060E070E004C040E855E260E070E082EEFA
:1023300095E00E94CB2CCF9108959091CC04492F29
:102340004F7050E0BA016F5F7F4F292F30E0E4E01B
:1023500035952795EA95E1F76217730759F0FA0169
:10236000E353FB4F808381E0890F8F70907F892B2F
:102370008093CC0408956EE770E082EE95E00E94B1
:1023800059060895A3E1B1E0E8ECF1E10C941F2EA9
:10239000E5E8F5E0712C8191882321F0739428E120
:1023A0007212F9CF66ED71E082EE95E00E946F2A1D
:1023B0004AE050E0672D82EE95E00E946C2B80E0B1
:1023C0000E947E0A0E94590B8E010E5F1F4FC12C86
:1023D000D12C7601C39466246A945C2C0E947728E1
:1023E0004B015C012091840530E0A0E1B7E20E943E
:1023F000952D9B01AC01C701B6010E94B72D20911C
:102400007B0530917C0540917D0550917E05620FE2
:10241000731F841F951F2091BB053091BC0540910F
:10242000BD055091BE05261737074807590718F410
:10243000F801608229C08C2D0E94B20961E070E031
:1024400080E090E00E94A628F80110820E94772880
:10245000681979098A099B09643F714081059105D2
:1024600040F40E94C809F8019081981778F780839A
:10247000EDCF50FE05C05D9841985E9A409A04C029
:102480005D9A419A5E9840982FEFC21AD20AE20AEA
:10249000F20A0F5F1F4F8FEFC816D104E104F10459
:1024A00009F09BCFCE019395FC01D82E7FEF68EC0D
:1024B0002E2F281B271510F051E056C0DE01129672
:1024C00051E02FEF41E03D91321710F0322F01C063
:1024D000452F5F5F5F3F11F0232FF5CF4193242FEE
:1024E00030E0A1E0B0E0AC0FBD1FA20FB31F5C93C2
:1024F000413079F0DE01A20FB31F5C93423049F006
:10250000AFEFBFEFAC0FBD1FA20FB31F6C934E3FD9
:1025100078F6A2E0B0E0AC0FBD1FA20FB31F7C9312
:102520004D3F30F6A3E0B0E0AC0FBD1FA20FB31FCC
:102530006C93BECF452F242F30E0FC01E20FF31F38
:102540006081AFEFB0E0AC0FBD1FA20FB31F2C91A5
:10255000621748F44150DC01A40FB11D2C91208377
:102560006C934111E8CF5F5F571520F3372D3695F7
:1025700020E0231770F4DC01A20FB11D4C91522F03
:10258000530FFC01E50FF11D50815C9340832E5FDA
:10259000F0CFF5E8EF2EF5E0FF2E8C01802F8D199E
:1025A000871598F4F801C1908F014AE050E06C2D36
:1025B00082EE95E00E94352B6CE282EE95E00E945F
:1025C000412AF701C1927F01E9CF82EE95E00E9496
:1025D000492A81E0CD5EDE4FEFE00C943B2E1F9246
:1025E0000F920FB60F9211241F932F933F934F9387
:1025F0005F936F937F938F939F93AF93BF93CF938B
:10260000DF93EF93FF93C0918600D0918700809174
:102610008704909188042091A904211155C09E013E
:10262000281B390B8091BF059091C005A091C10571
:10263000B091C20585FD02C036952795253C49E03D
:102640003407B8F140910A0150E060E070E02CE1FD
:10265000B695A795979587952A95D1F70097A105E7
:10266000B10521F481E090E0A0E0B0E08417950787
:10267000A607B707D8F480910A018F3FB9F040E070
:1026800080910A01481780F4842F90E0880F991FE9
:10269000FC01E757FB4F20813181FC01E55FFE4FD4
:1026A000318320834F5FECCF1092AA0410920A016D
:1026B0000BC02D3B82E0380720F080910A01803169
:1026C000D8F08FEF80930A01D0938804C0938704D9
:1026D000FF91EF91DF91CF91BF91AF919F918F913A
:1026E0007F916F915F914F913F912F911F910F902B
:1026F0000FBE0F901F90189510910A0181E0810F75
:1027000080930A01C9010E94DE08E12FF0E0EE0F7C
:10271000FF1FE757FB4F91838083D6CF83E08093E1
:1027200080008AE9809381008091BF0586FD05C005
:10273000809181008064809381008FEF9FEF909360
:1027400089008093880080916F00806280936F0081
:1027500008950E94300D8091D405843011F41092B8
:10276000D40508956F3018F086958058089589E053
:10277000689F802D11240895A0E0B0E0E2ECF3E121
:102780000C94262EC82F0E948328009138041091A3
:10279000390420913A0430913B046B017C01C01A4A
:1027A000D10AE20AF30A9701860149E8C41643E117
:1027B000D406E104F10410F010923C046093380454
:1027C0007093390480933A0490933B042091A904B8
:1027D0008FEF820F8230D8F5E0913C04EE2309F4AC
:1027E0004EC1E13011F482E0B8C1E03108F034C1EB
:1027F00081E08E0F80933C04F0E0E757FB4FC083ED
:10280000803109F0ACC1EBE8F4E0213029F4A1817A
:10281000A695A695808108C080819181A92FA69553
:10282000A695A69596958795A03148F4B0E090E0DE
:10283000AA0FBB1FA55FBE4F11969C938E9310925B
:10284000AA04329684E0E939F807F9F688C1233002
:1028500009F005C1E0913C04E11104C0CF3009F05A
:102860007EC10DC1E83148F481E08E0F80933C04B5
:10287000F0E0E857FB4FC08372C1E83109F0ECC0CB
:10288000C111EAC040E050E0ABE0CA01B3E0880FFC
:10289000991FBA95E1F7A49F9001A59F300D1124CF
:1028A000F901E757FB4F6081E1817E2F77707595C5
:1028B0006795FC01EE0FFF1FE55FFE4F718360839C
:1028C000F901E657FB4FB081B695B695B695E18113
:1028D000FE2FF295FF0FF07E6F2F6B2BE695E6959E
:1028E000E6957E2F777075956795FC01EE0FFF1FBB
:1028F000E35FFE4F71836083F901E557FB4FB081C1
:10290000B295B695B695B370C181DC2FDD0FDD0FA2
:102910006D2F6B2BC295C695C695C370E281E17091
:10292000EE0FEE0F7E2F7C2B75956795FC01EE0F59
:10293000FF1FE15FFE4F71836083F901E357FB4F97
:10294000B081B695E181FE2FF795FF27F7956F2FA0
:102950006B2BE6957E2F777075956795FC01EE0FD2
:10296000FF1FEF5EFE4F71836083F901E257FB4F5B
:10297000B081B295BF70E181FE2FF295F07F6F2F8D
:102980006B2BE295EF707E2F777075956795FC0144
:10299000EE0FFF1FED5EFE4F71836083F901E1577B
:1029A000FB4FB081BB1FBB27BB1FC181DC2FDD0FDD
:1029B0006D2F6B2BCC1FCC27CC1FE281E370EE0F69
:1029C0007E2F7C2B75956795FC01EE0FFF1FEB5E4C
:1029D000FE4F71836083F901EF56FB4FB081B695CE
:1029E000B695E181FE2FF295FF0FFF0FF07C6F2F60
:1029F0006B2BE695E6957E2F777075956795FC01B4
:102A0000EE0FFF1FE95EFE4F71836083F901EE5602
:102A1000FB4F20812295269527703181E32FEE0F01
:102A2000EE0FEE0F6E2F622B732F729576957770E7
:102A300075956795FC01EE0FFF1FE75EFE4F7183F2
:102A400060834F5F5F4F4230510509F01ECF809188
:102A50009F0483FF1092AA0410923C0480C024308B
:102A600009F07DC060913C0461110BC0C83AB1F41B
:102A7000109275051092740588EA0E94610681E043
:102A80006CC0613019F4C093370404C0623031F473
:102A9000C09336048C2F0E9461065AC0E091360420
:102AA0002E2F30E0220F331F462F50E0C90102962F
:102AB000841795073CF0633268F7FA01EA57FB4F39
:102AC000C083E8CF2D5F3F4F8C2F90E0609174055D
:102AD000709175054217530749F4982F8827862768
:102AE0009727909375058093740532C0681779070E
:102AF00069F580913704813049F5E13118F080E1C2
:102B000080933604F0903604CAE8D4E000E010E088
:102B10000F15D0F4FE013197808190E0982F88271F
:102B20002881822B63E0969587956A95E1F70E944C
:102B3000DE08F801EE0FFF1FE55FFE4F91838083F3
:102B40000F5F1F4F2296E4CF1092AA0410923C040C
:102B500080913C04882319F08F5F80933C04CDB7AB
:102B6000DEB7E8E00C94422EE82FF0E0E654FA4F8E
:102B7000E185E03150F4F894F0E0EE0FFF1FE55FDF
:102B8000FE4F8081918178940895E03121F0E13108
:102B900031F483E101C082E10E94C529089580E0FB
:102BA00092E00895A2E2B0E0E8EDF5E10C941C2E6D
:102BB0009E012F5F3F4F80E1D9011D928A95E9F771
:102BC00064E072E082EE95E029A33AA30E946F2AA6
:102BD0000E947C0B1D8A1E8A1F8A188E312C212C84
:102BE00000E0812C912C540170EC472E7DE9572E8A
:102BF00078E5672E75E3772EE0E5CE2EE3ECDE2E4A
:102C0000E12CF12C84EF91E0A0E0B0E08D8F9E8F5D
:102C1000AF8FB8A380EC97EFAAEBB7E3898F9A8FB9
:102C2000AB8FBC8F80EC9DE9A8E5B5E3898B9A8BCF
:102C3000AB8BBC8B82EE95E00E94832B892B09F431
:102C4000E1C082EE95E00E94B02B9C0133272C322C
:102C5000310509F442C0ACF42332310509F0ABC0B0
:102C600019821A821B821C821D821E821F82188674
:102C700019861A861B861C861D861E861F86188A44
:102C800060C02434310529F02335310509F4B2C080
:102C900092C064E482EE95E00E94412A2AE030E08E
:102CA00040EC5DE968E575E382EE95E00E94CF2A8D
:102CB0006CE282EE95E00E94412A2AE030E040EC8E
:102CC00057EF6AEB77E382EE95E00E94CF2A6CE241
:102CD00082EE95E00E94812AADCF0F5F043009F0AB
:102CE000A9CF29813A814B815C81A8EEB3E00E9493
:102CF000A42D698B7A8B8B8B9C8B2D813E814F8190
:102D000058850E94A42D698F7A8F8B8F9C8F29857F
:102D10003A854B855C852D8F3E8F4F8F58A32D852F
:102D20003E854F8558890E94A42D6B017C0160323D
:102D30003EE473078105910530F462E38CE10E9463
:102D40009F0900E077CF603345E77407810591055F
:102D500010F462E2F3CF60345CE9750781059105F8
:102D600010F466E2EBCF80E5C81683ECD806E104E8
:102D7000F10410F462E1E2CF90E6C9169AEED906AA
:102D8000E104F10410F465E1D9CFA0E7CA16A1E18E
:102D9000DA06A1E0EA06F10410F461E0CFCFB0EA70
:102DA000CB16B6E8DB06B1E0EB06F10410F463E005
:102DB000C5CF65E0C3CF10ED180F1A3008F03ACF39
:102DC000E1E0F0E0EC0FFD1F24E0029FE00DF11DBB
:102DD00011242081318142815381AAE0B0E00E9418
:102DE000A42D610F711D811D911D608371838283EC
:102DF000938320CF49885A886B887C88812C912CBA
:102E0000540118CF81149104A104B10489F4C301C1
:102E1000B2010E940E0A61E070E080E090E00E9442
:102E2000A6281D8A1E8A1F8A188E312C22242A94D5
:102E30008D8D9E8DAF8DB8A188169906AA06BB060A
:102E4000D0F40E94C8092D893E894F89588D280FDA
:102E5000311D411D511D2D8B3E8B4F8B588F3816C8
:102E600008F4382E821508F4282E3FEF831A930AAF
:102E7000A30AB30A56C0C301B20128EE33E040E012
:102E800050E00E94DB2DBA01A9012AE030E082EE79
:102E900095E00E94262B6CE282EE95E00E94412A8A
:102EA0004AE050E0632D82EE95E00E94352B6CE203
:102EB00082EE95E00E94412A6D897E898F89988DE6
:102EC000A50194010E94DB2DBA01A9012AE030E09E
:102ED00082EE95E00E94262B6CE282EE95E00E9445
:102EE000412A4AE050E0622D82EE95E00E94352BA7
:102EF0006CE282EE95E00E94812A4C0C5D1C6E1CF7
:102F00007F1C898D9A8DAB8DBC8D84159505A6058A
:102F1000B70520F449885A886B887C88812C912CCD
:102F2000540129893A894B895C89283E33404105FF
:102F3000510509F07FCEA296E2E10C94382EACE167
:102F4000B0E0E5EAF7E10C94262E0E9483286B019D
:102F50007C0181E00E947E0A14E703E0198361E0AE
:102F6000CE0101960E94DB0B009373050E94590B62
:102F70006AEF70E080E090E00E94A62880917305DF
:102F8000833089F482EE95E00E94832B892B59F4DB
:102F90000E9483286C197D098E099F096038734C43
:102FA000894C9140D8F280917305833009F44FC069
:102FB0008FE70E9477090E948A098983843511F07E
:102FC00083E05CC00E948A09109246058093470501
:102FD0000E948A092091460530914705280F311D2E
:102FE00030934705209346050E948A09809348053F
:102FF0000E948A0980934905813110F7F12C0F2D29
:1030000010E08091490590E0880F991F0817190773
:1030100040F40E948A09F801E65BFA4F8083F3943A
:10302000EECF80E7898361E0CE0101960E94DB0B41
:1030300083E0809373050E94590B62E370E080E0A7
:1030400090E00E94A62880917305833011F482E0FD
:1030500015C08FE70E9477090E948A09898380350D
:1030600009F0AECF0FE915E00E948A09F8018193BB
:103070008F01F5E00A3B1F07B9F781E06C96E8E0A5
:103080000C94422E80914505992787FD9095A92F94
:10309000B92FFC013196EB30F10508F066C0EC5C0D
:1030A000FF4F0C94532E62E778E082EE95E00E9489
:1030B0005D2A82E893E00E94300C6AE578E082EEB7
:1030C00095E00E945D2A65E378E082EE95E00E943B
:1030D0005D2A6BE078E082EE95E00E945D2A6AEE60
:1030E00077E082EE95E00E945D2A6DEB77E082EE5C
:1030F00095E00E945D2A67E977E082EE95E00E9404
:103100005D2A63E777E082EE95E00E945D2A6CE439
:1031100077E082EE95E00E945D2A82EE95E00E94C3
:10312000492A0E94700D21C06FE277E01AC06AE060
:1031300077E017C065EF76E014C066ED76E011C069
:1031400062E976E00EC06DE776E00BC068E676E0F7
:1031500082EE95E00E945D2A62E276E002C06CE0B9
:1031600076E082EE95E00E945D2A6AE070E080E001
:1031700090E00E94A62882EE95E00E94832B892B86
:1031800029F082EE95E00E94B02BF5CF0895ACE1D6
:10319000B0E0EDECF8E10C94262E909145059F3FB0
:1031A00009F023C1482F50E0FA013A97EF36F105B4
:1031B00008F00FC1E15CFF4F0C94532E61E172E007
:1031C000A0C06DE172E082EE95E00E946F2A85E773
:1031D00089838BE1EFE9F5E0DE01129601900D9213
:1031E0008A95E1F76CE1CE0101960E94DB0B0E940B
:1031F000590B83E08093730568EC70E080E090E009
:103200000E94A62880917305843009F0E2C08FE700
:103210000E9477090E948A098983853509F0D9C0FF
:103220006DEE74E082EE95E00E945D2A6FEC74E032
:1032300082EE95E00E945D2A61EB74E096C065E342
:1032400072E082EE95E00E946F2A89E6898361E050
:10325000CE0101960E94DB0B0E94590B83E0809304
:10326000730568EC70E080E090E00E94A6288091F1
:103270007305843009F0ADC08FE70E9477090E9482
:103280008A0989838E010E5F1F4F7E014DE1E40E96
:10329000F11C0E948A09F80181938F01EE15FF0548
:1032A000C1F78BE1FE013296AFE9B5E001900D92D6
:1032B0008A95E1F78981893409F08BC063E974E06C
:1032C00082EE95E00E945D2A65E774E082EE95E06B
:1032D0000E945D2A67E574E048C06FE472E082EE08
:1032E00095E00E946F2A8EEF8093450572C0805250
:1032F0008750805390914805981708F066C06EE596
:1033000072E082EE95E00E946F2A63C084E18093B0
:10331000450560E274E029C085E18093450569EECA
:1033200073E023C086E18093450562EB73E01DC026
:1033300087E18093450568E673E017C088E18093D4
:10334000450567E573E011C089E18093450563E4B5
:1033500073E00BC08AE1809345056EE273E005C01F
:103360008BE18093450566E073E082EE95E00E9474
:103370005D2A2FC06CEE72E082EE95E00E945D2A1D
:103380008091AD0591E01DC066ED72E082EE95E0A2
:103390000E945D2A8091AD0592E013C061EC72E05D
:1033A00082EE95E00E945D2A8091AD0594E009C00F
:1033B00066EA72E082EE95E00E945D2A8091AD059A
:1033C00098E089278093AD058FEF809345050E9493
:1033D000111082EE95E00E94832B892B09F45BC1CA
:1033E00082EE95E00E94B02BF4CF0E94101188234A
:1033F00009F451C18091DF04811104C08FEF8093E3
:10340000450541C140E050E060E070E080EE94E0AE
:103410000E94CA2E40914505042F112707FD1095E3
:10342000212F312FF8013197EB31F10508F01BC145
:10343000E255FF4F0C94532E552747FD5095209190
:10344000480530E0241735070CF40DC18B019C01B1
:1034500001501109210931090032110521053105F9
:1034600058F0C0904905EBE4F5E0F12CD12CA8E22E
:10347000EA2E415051090FC0FA01E156FA4F61504E
:103480006083D9C0DF0111972C9130E024173507F4
:1034900029F0F3943296FC10F5CFCBC00E2D10E03E
:1034A00020E030E0061717072807390741F420818C
:1034B000DA01A156BA4F11962C93DD24D394E394EC
:1034C000E8CF6F3F71058105910511F008F0CBC081
:1034D0006093B705B0C06F3F71058105910511F08C
:1034E00008F0C1C06093B805A6C06F3F71058105A3
:1034F000910511F008F0B7C06093B9059CC0209108
:10350000E00420622037E9F440E050E060E070E041
:1035100081EE94E00E94CA2E9B01AC01DC01CB013C
:103520000197A109B1090897A105B10508F0AEC03E
:10353000A4EDB0E30E94A42D6A5E7C4A8A46954EB3
:1035400024C02636E9F440E050E060E070E081EE0F
:1035500094E00E94CA2E9B01AC01DC01CB010197D3
:10356000A109B1090797A105B10508F08FC0A8EA24
:10357000B1E60E94A42D645E7C438E46944E05C045
:10358000611571058105910579F08B019C01005C45
:103590001D49284535430130FAE51F07F2E62F079C
:1035A000F2E03F0708F05FC06093AF057093B0058D
:1035B0008093B1059093B2053EC06F3F71058105C0
:1035C000910511F008F04FC06093B30534C08B0132
:1035D0009C0101501109210931090F3F11052105F5
:1035E000310508F040C06093B40525C08B019C01F3
:1035F000045C1940210931090D344DE114072105FE
:10360000310528F47093B6056093B50514C06115B3
:1036100071058105910521F48FEF8093AE050BC0F4
:103620006134710581059105F0F461506093AE0538
:1036300002C0DD20C1F08091DE0481111AC08091AA
:103640007F0590918005A0918105B091820501963A
:10365000A11DB11D80937F0590938005A0938105E6
:10366000B093820506C060E772E082EE95E00E94AA
:103670006F2A0E9406118FEF809345056AE082EE63
:1036800095E00E94812A0E94111005C061E070E05F
:1036900080E090E07ACF6C96E8E00C94422E6AE5E8
:1036A00072E082EE95E00E945D2A62E472E082EEB2
:1036B00095E00E945D2A82EE95E00E94832B892B83
:1036C00031F082EE95E00E94B02B0E94C7180E9454
:1036D0009F17823029F0833051F46DE072E002C010
:1036E00064E272E082EE95E00E945D2A08958FEF19
:1036F000809345051092DE040E94111080914505CB
:103700008E3F69F082EE95E00E94832B892BB1F306
:1037100082EE95E00E94B02B0E94C718EFCF08956B
:103720000F931F93109145051F3F09F0D2C08934B4
:1037300009F457C000F5883309F469C058F48033A0
:1037400009F477C008F061C08B3109F440C08132C0
:10375000B1F1B9C0813409F487C030F4893309F478
:1037600066C0803461F1AFC0823409F48EC0863403
:1037700009F448C0A8C0823609F487C078F48835B7
:1037800031F128F48235C1F18335E1F09CC08A35EE
:1037900009F494C0813609F467C095C0823761F19D
:1037A00028F4863679F18936E1F08DC0883779F0D2
:1037B0008A3709F483C0833709F085C003C061E10B
:1037C00072E015C00E94410D6EE872E004C00E94D4
:1037D0004A0D68EA72E082EE95E00E946F2A8EEF51
:1037E00070C00E947A060E94BF0667EC72E082EE0B
:1037F00095E00E946F2A67C081E00E94DF0660EEBC
:1038000072E0F5CF0E94BB105EC080535AC06AEFD1
:1038100071E082EE95E00E945D2A90919E0588E01D
:10382000890F8871977E892B80939E051AC089E045
:1038300048C067EE71E082EE95E00E945D2A8091BB
:10384000BF059091C005A091C105B091C20520E1CE
:1038500082278093BF059093C005A093C105B093C4
:10386000C205109345052FC061ED71E082EE95E031
:103870000E945D2A8091BF059091C005A091C1056D
:10388000B091C20540E4842710C060EC71E082EE84
:1038900095E00E945D2A8091BF059091C005A0919E
:1038A000C105B091C20520E282278093BF059093A5
:1038B000C005A093C105B093C20502C00E944F1B72
:1038C0008FEF80934505809145058E3F09F0D4C068
:1038D000DDC00E941011882309F4D8C08091DF0454
:1038E000811104C08FEF80934505C6C040E050E0D1
:1038F00060E070E080EE94E00E94CA2E00914505E1
:10390000112707FD1095212F312FF8013197E9304C
:10391000F10508F0B4C0E753FF4F0C94532E8B0110
:103920009C01015C1D49284535430F3F194522463E
:10393000324008F0A4C060937B0570937C058093AF
:103940007D0590937E0577C060937F057093800519
:10395000809381059093820581E08093DE046BC0A3
:10396000683071058105910508F089C06093830571
:1039700062C08B019C0101501109210931090A30F3
:1039800011052105310508F07AC06093840553C004
:1039900061EB71E080EE94E00E94043010E000974B
:1039A00099F00E94DE2F009779F0183130F4E12F62
:1039B000F0E0EA58FA4F87871F5F61EB71E080E023
:1039C00090E00E940430EBCF1831A8F5E12FF0E031
:1039D000EA58FA4F17861F5FF7CF653071058105EA
:1039E000910508F04CC060939D0525C08B019C019A
:1039F0000150110921093109063011052105310550
:103A0000F0F520919E05287F262B20939E0513C05C
:103A10008B019C0101501109210931090115124C3A
:103A20002140310560F560937705709378058093A8
:103A3000790590937A058091DE04811113C08091FD
:103A40007F0590918005A0918105B0918205019636
:103A5000A11DB11D80937F0590938005A0938105E2
:103A6000B09382050E9406118FEF809345056AE0AE
:103A700082EE95E00E94812A0E94421807C060E70A
:103A800072E082EE95E00E946F2AECCF1F910F91B9
:103A900008958FEF809345051092DE040E9442182E
:103AA000809145058E3F69F082EE95E00E94832B60
:103AB000892BB1F382EE95E00E94B02B0E94901BFF
:103AC000EFCF6AE070E080E090E00E94A62882EEEE
:103AD00095E00E94832B892B29F082EE95E00E94CD
:103AE000B02BF5CF0895CF93C82F682F82EE95E0C5
:103AF0000E94DD2B90916A059C2790936A05CF91D7
:103B00000895A1E0B0E0E7E8FDE10C942C2E998344
:103B10000E94731D9981892F0E94731D2196E2E0F6
:103B20000C94482E1F93CF93DF93182FEB01109224
:103B30006A0565EB70E082EE95E00E94590662E648
:103B400070E082EE95E00E945906812F0E94731D5D
:103B5000CE010E94811DDF91CF911F910895609148
:103B60006A0582EE95E00E94DD2B0895A1E2B0E0A7
:103B7000ECEBFDE10C94282E7B018A018C3009F4DA
:103B800053C108F040C0863009F4BCC018F583303A
:103B900009F491C070F4813009F472C0823009F0E8
:103BA00048C26BE170E082E00E94921D0FE915E0CF
:103BB00078C0843009F487C0853009F03AC260913A
:103BC000490570E0660F771F85E00E94921D0AE4A8
:103BD00015E086C0893009F4A7C070F4873009F475
:103BE0009BC0883009F025C261E070E088E00E9447
:103BF000921D8091D40523C28A3009F4CAC08B304B
:103C000009F4F2C016C28A3609F475C1D8F48736B1
:103C100009F43AC138F4853609F40EC1863609F440
:103C20001FC107C2883609F437C1893609F001C2BD
:103C300061E070E089E60E94921D0E947A060E946F
:103C4000BF06F5C18D3609F4D4C138F48B3609F4BA
:103C500091C18C3609F49AC1ECC18E3609F4DCC1ED
:103C6000873C09F0E6C161E070E087EC0E94921D9C
:103C700081E00E94731D0E94AF1D10926B05E3C18D
:103C800069E270E081E00E94921D06E715E0F8010C
:103C900081918F010E94731DF5E00F391F07B9F75D
:103CA000D0C1F80181918F010E94731DF5E00A3B9C
:103CB0001F07B9F7C6C161E070E083E00E94921D62
:103CC0000E949F17BCC161E070E084E00E94921DD9
:103CD00081E00E94731D0E94AF1D0E94D215B3C1E6
:103CE0008091490590E0880F991F98012A5435402A
:103CF0002817390708F0A5C1F80181918F010E94AA
:103D0000731DEECF62E070E086E00E94921D82E8B3
:103D100093E00E94811D95C161E070E087E00E9400
:103D2000921D809148058BC186E6898361E0CE01B2
:103D300001960E94DB0B0E94590B83E08093730570
:103D400068EC70E080E090E00E94A6288091730506
:103D50008430D9F48FE70E9477090E948A09898309
:103D6000863469F460E270E089E00E94921D10E2FE
:103D70000E948A090E94731D1150D1F762C161E04F
:103D800070E089E00E94921D52C161E070E089E01C
:103D900053C169E170E08AE00E94921D82E0809345
:103DA000BA05209172058091BF059091C005A09140
:103DB000C105B091C205222311F0806801C08F7740
:103DC0008093BF059093C005A093C105B093C20531
:103DD0000AEB15E0F80181918F010E94731DF5E057
:103DE000033D1F07B9F72DC161E270E08BE00E942F
:103DF000921D8091AA048F3F39F08091AA0491E02E
:103E0000980F9093AA0402C08091AA040E94731D87
:103E100010E0812F0E94B4150E9409090E94811DA3
:103E20001F5F1031B1F70DC161E070E08CE00E94BE
:103E3000921D8091D30503C161E070E085E60E9488
:103E4000921D89E2E816F10409F0F8C0D801E6E70E
:103E5000F5E08D91819385E0EF39F807D1F7E7C060
:103E600061E070E086E60E94921DEBE1EE16F1043F
:103E700009F0E4C0D801EFE9F5E08D91819385E088
:103E8000EA3BF807D1F7D3C061E070E087E60E9413
:103E9000921D0E94410DCBC061E070E088E60E9457
:103EA000921D85E789838BE1EFE9F5E0DE0112964B
:103EB00001900D928A95E1F76CE1CE0101960E9486
:103EC000DB0B0E94590B83E08093730560E273E083
:103ED00080E090E00E94A62880917305843009F06C
:103EE000ADC08FE70E9477090E948A0989838535D2
:103EF00009F0A4C09CC061E070E08AE60E94921DB7
:103F000089E6898361E0CE0101960E94DB0B0E9465
:103F1000590B83E08093730560E273E080E090E0EA
:103F20000E94A62880917305843009F087C08FE72E
:103F30000E9477090E948A0989838E010E5F1F4FB4
:103F40007E01EDE1EE0EF11C0E948A09F8018193D9
:103F50008F01EE15FF05C1F78BE1FE013296AFE947
:103F6000B5E001900D928A95E1F78981893409F0D5
:103F700065C05DC061E070E08BE60E94921DF801B3
:103F800080818093D4050E944A0D51C061E070E0A9
:103F90008CE60E94921DF0E2EF16F10461F487E6D0
:103FA000898380E2F801DE01129601900D928A95D4
:103FB000E1F761E203C087E4898361E0CE01019605
:103FC0000E94DB0B0E94590B83E0809373056CE425
:103FD00074E080E090E00E94A62880917305843010
:103FE00069F58FE70E9477090E948A09873431F5C5
:103FF0001EC061E070E08DE60E94921D89E1E81626
:10400000F104E1F4D801EAEBF5E08D91819385E0CC
:10401000E33DF807D1F70BC061E070E08EE60E9447
:10402000921DF80180818093D3050E942B0D81E0C1
:1040300006C061E070E08AEC0E94921D80E00E9460
:10404000731D0E94AF1DA196E6E00C94442EA0E0E3
:10405000B0E0EDE2F0E20C94262ECAECD3E014E6D8
:1040600006E035E0F32E44E0E42E53E0D52E62E086
:10407000C62E82EE95E00E94832B892B09F49BC00B
:1040800082EE95E00E94B02B282F8093350440915A
:10409000340450E04730510560F7FA01EE52FF4F0B
:1040A0000C94532E853B29F781E080933404E1CFB3
:1040B000823609F07DC0C0923404DBCF8093330494
:1040C00080933204D0923404D4CF9C0133273093B0
:1040D0003104209330049091320498279093320455
:1040E000E0923404C6CF382F2227409130045091FB
:1040F0003104242B352B30933104209330049091DC
:104100003204982790933204F09234042536310516
:1041100008F4AFCF61E070E08CEC0E94921D81E06A
:104120000E94731D0E94AF1D43C020912E04309148
:104130002F04F901E653FC4F8083909132049827B5
:1041400090933204C901019690932F0480932E041A
:1041500020913004309131048217930708F489CFFD
:104160000093340486CF8091320482130BC0609197
:104170002E0470912F044AEC53E0809133040E9486
:10418000B61D0DC062E070E08BEC0E94921D809124
:1041900033040E94731D80916A050E94731DFE0105
:1041A000812F11928A95E9F710922F0410922E0414
:1041B000109234045ECFCDB7DEB7E8E00C94422E07
:1041C00081E080936B0580916B05882349F082EE36
:1041D00095E00E94832B892BB1F30E942720F3CF17
:1041E0000895AAE2B0E0E7EFF0E20C94242E0E94DA
:1041F00077286B017C0181E00E947E0A82EE95E0C7
:104200000E94832B892B29F082EE95E00E94B02B2F
:10421000F5CF5E98409811E072E6B72EE9E2AE2E37
:1042200003E00E9477286C197D098E099F09693C7B
:10423000710581059105E0F11123D1F10E947728E4
:104240006B017C015D9A419A80ED97E00E94A8077E
:10425000B982E6E7F5E0DE0112968A2D01900D9213
:104260008A95E1F76AE2CE0101960E94DB0B5D9828
:10427000419880E090E00E94A807009373050E9497
:10428000590B62E370E080E090E00E94A6288091E4
:104290007305843061F4009373058FE70E947709FA
:1042A0000E948A0911E0823419F410E001C011E083
:1042B00083E10E949C29892BA1F411E012C05E9A2F
:1042C000409A5D9A419A82EE95E00E94B02B8D3023
:1042D0009105B9F06CF40A97A1F05E9840985D984A
:1042E000419882EE95E00E94832B892B41F799CF6C
:1042F0008332910579F08234910579F70E94E020AC
:10430000ECCF62EB71E082EE95E00E945D2A0E94A4
:10431000491DE3CF0E94D215E0CF8F929F92AF92BA
:10432000BF92CF92DF92EF92FF921F93CF93DF93D2
:1043300083E10E949C29892B09F089C068EC70E018
:1043400080E090E00E94A62880E090E00E94A8070C
:104350000E9477284B015C016B017C0180ECC80E48
:1043600082E1D81EE11CF11C0E9477286C157D05A6
:104370008E059F0530F483E10E949C29892BA1F3CF
:1043800064C083E10E949C29892B09F05EC080ED06
:1043900097E00E94A8070E9477286B017C01D0E07B
:1043A000C1E088E4880E86E2981EA11CB11C11E0D1
:1043B00083E10E949C29892B21F58C149D04AE0475
:1043C000BF0430F480ED97E00E94A807D1E0F0CF61
:1043D0000E9477286C197D098E099F09693C710537
:1043E0008105910528F30E9477286B017C01C12784
:1043F00019F080ED97E002C080E090E00E94A807ED
:10440000D7CF80E090E00E94A807DD23B9F080912B
:10441000D30590E0019665E070E00E94C72D80937F
:10442000D3050E942B0D0E94A9130E944A0D64EF30
:1044300071E080E090E00E94A62809C080E00E9420
:10444000DF060E94C2110E94410D0E94F120DF91FF
:10445000CF911F91FF90EF90DF90CF90BF90AF90E2
:104460009F908F900895CF92DF92EF92FF9280E01D
:104470000E94DA070E94B10761E086E00E943029BD
:1044800061E085E00E94302961E08EE00E943029E1
:1044900061E08FE00E94302960E083E10E943029D2
:1044A00060E088E00E94302961E088E00E9469298C
:1044B0000E949F0740E052EC61E070E082EE95E0E0
:1044C0000E94CB2C0E94A9130E944A0D0E948E13B9
:1044D0008FEF8093AA040E94C60778940E947728E1
:1044E0006B017C018091AA048F3F59F40E947728C8
:1044F0006C197D098E099F09603D77408105910502
:1045000088F380ED97E00E94A80761E083E10E94B4
:1045100069295E9A409A82EE95E00E94832B892B4E
:1045200029F082EE95E00E94B02BF5CF6DEF72E09E
:1045300082EE95E00E943E2A82E893E00E94300CD1
:1045400064E173E082EE95E00E943E2A4AE050E08A
:1045500067E070E082EE95E00E940E2B62E370E06F
:1045600080E090E00E94A62882EE95E00E94832BD6
:1045700004970CF182EE95E00E94B02B82349105F5
:10458000D1F482EE95E00E94B02B8E34910599F41F
:1045900082EE95E00E94B02B8434910561F482EEA6
:1045A00095E00E94B02B819731F480E090E00E946A
:1045B000A8070E94F12040917705509178056091FD
:1045C000790570917A05DB01CA010197A109B1094A
:1045D0000497A105B10568F44093A904433029F478
:1045E00040EA56E861E070E004C040E052EC61E06F
:1045F00070E082EE95E00E94CB2C0E948D215E98A7
:10460000409880E090E00E94A8070E948E131092CC
:10461000C5048091BF0583FF11C080918B0588235D
:1046200051F080919205882331F08091990588237B
:1046300011F087E001C085E08093C50480E00E940E
:104640007E0A8091C6040E94B2090E94590B109202
:104650003F0410923E0410923D04F12C8091D40549
:104660008F15B0F062E370E080E090E00E94A62831
:1046700080ED97E00E94A80762E370E080E090E0A0
:104680000E94A62880E090E00E94A807F394E6CF5D
:1046900080919E0584FF08C0982F987181E0983121
:1046A00009F080E00E947E118FE00E94DA07FF90FF
:1046B000EF90DF90CF900895EF92FF920F931F93AA
:1046C000CF93DF938C016EE770E082EE95E00E945D
:1046D0005906E801F12CF0E2EF2E8E0188818D570A
:1046E000823048F46DE770E082EE95E00E94590652
:1046F00088818E2588832196F801608182EE95E07D
:104700000E94DD2BF394F9E0FF12E7CF6EE770E033
:1047100082EE95E00E945906CDB7DEB7E6E00C9434
:10472000442EA9E0B0E0E7E9F3E20C942C2E90913E
:10473000C70491110EC09EEF99838A836B8350E06A
:10474000559547954C832D83198618861F821E82A6
:104750002EC04091CC04842F90E0B4E095958795CD
:10476000BA95E1F7242F2F7030E08217930719F1E3
:104770008DEF89831B82FE01349650E0842F90E0F8
:10478000A4E095958795AA95E1F7242F2F7030E046
:104790008217930749F0DC01A353BB4F8C9181939F
:1047A000405F5F5F563051F74093CC045A83CE018F
:1047B00001960E945C238091C70490E0019666E018
:1047C00070E00E94C72D8093C7042996E2E00C9404
:1047D000482EA0E0B0E0EFEEF3E20C94252E6C0141
:1047E0006EE770E082EE95E00E9459068601E12CAA
:1047F000F12CC0E0D0E030E2B32EF801608183E814
:10480000860F823078F46DE770E082EE95E00E94CA
:104810005906F80160816B2570E082EE95E00E94F8
:10482000590604C082EE95E00E94DD2BE114F104EC
:1048300059F0F80180819E01280F311DC901C92F4F
:10484000DD27C80FD91FDD273FEFE31AF30A89E000
:10485000E816F10459F028E0E216F10421F48C2F57
:104860008095F60180870F5F1F4FC7CFCDB7DEB7AA
:10487000E9E00C94412EA9E0B0E0E1E4F4E20C940C
:104880002C2EE82F362F8091C70490E0019664E229
:1048900070E00E94C72D8093C70458E9598350E106
:1048A0005A83813089F048F08230B9F08330D9F4EE
:1048B0008B8381EF8C833D8319C085E08B8381EFEF
:1048C0008C832F5F2D8312C08B8381EF8C8384E6D2
:1048D000489FA00111245D8309C084E08B8381EF90
:1048E0008C83ED8303C00E94BB1104C0CE010196EE
:1048F0000E94E9232996E2E00C94482EA2E0B0E061
:10490000E4E8F4E20C94212E182F762E2A834983B2
:104910000E9483286B017C018091DD048090C80493
:104920009090C904A090CA04B090CB042A81498118
:104930008823C1F0D701C60188199909AA09BB09C2
:104940004C015D0191EE89169EE29906A104B10425
:1049500020F1241708F4422F202F672D812F0E9469
:104960003B2413C0D701C60188199909AA09BB09BC
:104970004C015D0191E3891695E79906A104B10404
:1049800060F0672D812F0E949123C092C804D092BD
:10499000C904E092CA04F092CB042296EDE00C9494
:1049A0003D2EA2E2B0E0E7EDF4E20C94222E8CE082
:1049B0000E94990981110FC06CE173E082EE95E0CD
:1049C0000E946F2A5E9A409A80E00E947E0A0E94AE
:1049D000590B5E98409882EE95E00E94832B892BBC
:1049E00001F182EE95E00E94B02B9091A9049923E9
:1049F00019F00E94BC13EFCF40913E0450E09A01A1
:104A00002F5F3F4F2F71332760913F0470E02617CF
:104A1000370709F3FA01E75BFB4F808320933E04DD
:104A2000DACF80917305843009F086C00E94832814
:104A3000611571058105910549F06093B704709384
:104A4000B8048093B9049093BA040CC081E090E05C
:104A5000A0E0B0E08093B7049093B804A093B904A9
:104A6000B093BA048091AD049091AE0481609093AC
:104A7000AE048093AD0483E0809373058FE70E94BA
:104A8000770909E614E00E948A09F80181938F01F1
:104A9000F4E002371F07B9F720917204809169048E
:104AA000982F922796FF3BC090E492279093720430
:104AB000982F98739833F1F410E0212F30E0809113
:104AC0006904877090E0821793074CF11F5F209173
:104AD0009E05812F90E0FC01E759FB4F24FF04C0A5
:104AE00080810E949D11E9CF608182EE95E00E9455
:104AF000DD2BE3CF8F7399F480916A048093B60421
:104B000080916B048093B40480916C048093B3040F
:104B100080916F0490E09093AC048093AB048091FB
:104B20003D04813019F482E080933D0480913D047E
:104B3000833011F410923D040E9483286B017C01A4
:104B40008091AF049091B004A091B104B091B204EF
:104B50000097A105B105C9F0A7019601281B390BE3
:104B60004A0B5B0BDA01C901883B9B40A105B105EB
:104B700060F00E94C8098093B5041092AF041092AF
:104B8000B0041092B1041092B2048091BB049091D1
:104B9000BC04A091BD04B091BE0446015701881A1F
:104BA000990AAA0ABB0A86E795E00E94F4078616CE
:104BB0009706A806B90608F4A9C0C092BB04D09213
:104BC000BC04E092BD04F092BE040E94570680919E
:104BD000AA048830A0F08091BF059091C005A091F3
:104BE000C105B091C2055CE1B695A79597958795EB
:104BF0005A95D1F7892B8A2B8B2B09F0A2C1809172
:104C0000AA048F5F8093AA048091B7049091B8049E
:104C1000A091B904B091BA040097A105B105F1F0D3
:104C2000C81AD90AEA0AFB0A86E795E00E94F40747
:104C30006C157D058E059F0508F008C18091BF05A4
:104C400084FD04C080ED97E00E94A8071092B7048D
:104C50001092B8041092B9041092BA0490917204A0
:104C6000907C9093720450913E0480913F04209177
:104C70003D04581709F407C1223009F004C19058C7
:104C800090937204E0919E05E770F0E0E658FC4FC7
:104C90006081693008F0DFC0615040E04613DDC03C
:104CA00080933F0487E3840F90917204892B809353
:104CB00072044093400483E080933D045D9A419ADE
:104CC000809183059091C50491112CC10E94790AAD
:104CD0008091C6040E94B209E0919E05E770F0E061
:104CE000E658FC4F608182E794E00E94940BE091CB
:104CF000C604EF5FE093C604E83109F41FC1F0E099
:104D0000EA58FA4F8785882309F418C10E94030CDA
:104D1000813069F580919E05887149F18091AD04DB
:104D20009091AE04880F991F9093AE048093AD04C8
:104D300083E0809373050E94590B0E94832860933F
:104D4000AF047093B0048093B1049093B204672BC6
:104D5000682B692B61F481E090E0A0E0B0E08093E3
:104D6000AF049093B004A093B104B093B2048091C7
:104D70009E0584FF1FC08091AD049091AE048E7F8C
:104D80000E942A09182F6091AB048091B6040E94FA
:104D9000B213482F612F8091B50449A30E94B2132A
:104DA0000091D405282F49A16091B3048091B404E7
:104DB0000E947E245D9841988091C3048130C1F0A7
:104DC00018F08230B1F1CBC083E10E949C29892B7D
:104DD00009F0C5C081E08093C3040E9477286093E6
:104DE000BF047093C0048093C1049093C204B7C001
:104DF00083E10E949C29892B31F50E947728C0907D
:104E0000BF04D090C004E090C104F090C2046C19BB
:104E10007D098E099F09693E73408105910508F45B
:104E20009EC082E08093C30480ED97E00E94A807B3
:104E300096C083E10E949C29892B09F490C080E0F0
:104E400090E00E94A8071092C30489C080E090E01F
:104E50000E94A80703CF68E020CF851709F420CF70
:104E60004F5F242F30E090E0F901EE58FB4FDC015A
:104E7000A75BBB4F7C917083F901E05CFB4F7083B3
:104E800001968F710BCF2430B1F42091400481E45E
:104E900094E0A3E7B4E0FC013E2F381B321718F46E
:104EA00031913D93F9CF87E3820F90917204892B62
:104EB0008093720400CF8091C304823059F49160D2
:104EC000909372045E9A409A8E010F5F1F4FF12CEF
:104ED000B80111C05E98409880913D04811103C0D3
:104EE00081E080933D0480913D04833069F784E044
:104EF00080933D04E9CF8F2D69A37AA30E94B41556
:104F0000F801819391938F01F39469A17AA1F0E163
:104F1000FF12F1CF80919E0543E754E087700E9415
:104F20007908CCCE882309F4D1CE2091C40431E095
:104F3000320F3093C4042913C9CE0DC01092C60499
:104F4000E5CE8091AA04883011F45E9A409A89E0F7
:104F50008093AA04DBCE1092C4048150B7CEA296EF
:104F6000ECE00C943E2E8230E8F4E82FF0E0EE0FF7
:104F7000FF1FEB52FA4F71836083813041F08091C3
:104F800069008C7F842B80936900E89A0895809152
:104F90006900440F551F440F551F837F842B809356
:104FA0006900E99A08951F920F920FB60F9211248B
:104FB0002F933F934F935F936F937F938F939F9321
:104FC000AF93BF93EF93FF938091D5059091D60552
:104FD000892B29F0E091D505F091D6050995FF912F
:104FE000EF91BF91AF919F918F917F916F915F9161
:104FF0004F913F912F910F900FBE0F901F901895DA
:105000001F920F920FB60F9211242F933F934F933D
:105010005F936F937F938F939F93AF93BF93EF9320
:10502000FF938091D7059091D805892B29F0E091C5
:10503000D705F091D8050995FF91EF91BF91AF91F8
:105040009F918F917F916F915F914F913F912F91A0
:105050000F900FBE0F901F9018951F920F920FB6D2
:105060000F9211242F933F938F939F93AF93BF93EE
:105070008091DA059091DB05A091DC05B091DD050A
:105080003091D90523E0230F2D3720F40196A11D7F
:10509000B11D05C026E8230F0296A11DB11D209366
:1050A000D9058093DA059093DB05A093DC05B093D6
:1050B000DD058091DE059091DF05A091E005B091BE
:1050C000E1050196A11DB11D8093DE059093DF05DA
:1050D000A093E005B093E105BF91AF919F918F91AF
:1050E0003F912F910F900FBE0F901F9018952FB7E3
:1050F000F8946091DA057091DB058091DC05909160
:10510000DD052FBF08953FB7F8948091DE0590919B
:10511000DF05A091E005B091E10526B5A89B05C08B
:105120002F3F19F00196A11DB11D3FBF6627782FB3
:10513000892F9A2F620F711D811D911D42E0660F0C
:10514000771F881F991F4A95D1F70895CF92DF9254
:10515000EF92FF92CF93DF936B017C010E94832833
:10516000EB01C114D104E104F10479F00E94832819
:105170006C1B7D0B683E7340A0F381E0C81AD10818
:10518000E108F108C851DC4FECCFDF91CF91FF90DF
:10519000EF90DF90CF900895789484B5826084BDBD
:1051A00084B5816084BD85B5826085BD85B581602B
:1051B00085BDEEE6F0E0808181608083E1E8F0E08B
:1051C0001082808182608083808181608083E0E8BA
:1051D000F0E0808181608083E1EBF0E08081846099
:1051E0008083E0EBF0E0808181608083EAE7F0E09B
:1051F00080818460808380818260808380818160FF
:1052000080838081806880831092C10008958330FC
:1052100081F028F4813099F08230A1F00895863031
:10522000A9F08730B9F08430D1F4809180008F7D6F
:1052300003C0809180008F7780938000089584B5AB
:105240008F7702C084B58F7D84BD08958091B000B2
:105250008F7703C08091B0008F7D8093B000089558
:10526000CF93DF9390E0FC01ED50F44F2491FC01CB
:10527000E95FF34F8491882349F190E0880F991FEB
:10528000FC01E15DF34FA591B4918B5D934FFC015F
:10529000C591D4919FB7611108C0F8948C91209565
:1052A00082238C93888182230AC0623051F4F8945F
:1052B0008C91322F309583238C938881822B888325
:1052C00004C0F8948C91822B8C939FBFDF91CF9177
:1052D0000895A1E0B0E0EFE6F9E20C942A2E282F21
:1052E00030E0F901E152F44F8491F901ED50F44FAF
:1052F0001491F901E95FF34F04910023C9F0882369
:1053000021F069830E9407296981E02FF0E0EE0F08
:10531000FF1FEB5DF34FA591B4919FB7F8948C916B
:10532000611103C01095812301C0812B8C939FBF15
:105330002196E4E00C94462ECF93DF93282F30E0A3
:10534000F901E152F44F8491F901ED50F44FD491F9
:10535000F901E95FF34FC491CC2391F081110E94D0
:105360000729EC2FF0E0EE0FFF1FE55EF34FA5914C
:10537000B4912C912D2381E090E021F480E002C0D3
:1053800080E090E0DF91CF9108958E3008F08E504C
:10539000877020919D0190E4299F90011124822B18
:1053A00080937C0080917A00806480937A00809161
:1053B0007A0086FDFCCF809178002091790090E002
:1053C000922B0895A0E0B0E0E8EEF9E20C94262ECE
:1053D0006C017A01EB01E60EF71E00E010E0CE153D
:1053E000DF0561F06991D601ED91FC910190F081AA
:1053F000E02DC6010995080F191FF1CFC801CDB7DF
:10540000DEB7E8E00C94422E6115710589F0DB01EE
:105410000D900020E9F7AD0141505109461B570B93
:10542000DC01ED91FC910280F381E02D0995089556
:1054300080E090E00895EF92FF920F931F93CF9337
:10544000DF938C01FB01C0E0D0E064917F018FEF1E
:10545000E81AF80A662361F0D801ED91FC910190F9
:10546000F081E02DC8010995C80FD91FF701EDCFD4
:10547000CE01CDB7DEB7E6E00C94442E0E94042A9C
:105480000895DC01ED91FC910190F081E02D0995EA
:1054900008950F931F93CF93DF93EC016DE00E946B
:1054A000412A8C016AE0CE010E94412A800F911F9F
:1054B000DF91CF911F910F9108950F931F93CF9379
:1054C000DF93EC010E941B2A8C01CE010E94492A25
:1054D000800F911FDF91CF911F910F9108950F932E
:1054E0001F93CF93DF93EC010E94042A8C01CE011D
:1054F0000E94492A800F911FDF91CF911F910F9138
:1055000008950F931F93CF93DF93EC010E94412ADC
:105510008C01CE010E94492A800F911FDF91CF910B
:105520001F910F910895A1E2B0E0E9E9FAE20C942D
:10553000222E7C01C42EE52FCB01D22E19A221E010
:105540002D1510F02AE0D22E8E010F5D1F4F8D2CED
:10555000912CA12CB12C6C2D7E2FA50194010E94C1
:10556000DB2D8C2DD29E80191124015011098A3017
:1055700010F4805D01C0895CF8018083211531053C
:105580004105510521F0C22EE32FCA01E4CFB80135
:10559000C7010E94042AA196ECE00C943E2EA0E0E4
:1055A000B0E0E5EDFAE20C94262EEC016A017B01F5
:1055B0002115310541F4E881F9810190F081E02D58
:1055C000642F09951DC02A303105A9F477FF12C058
:1055D0006DE20E94412A8C0144275527BA014C19DB
:1055E0005D096E097F092AE0CE010E94932A800F8F
:1055F000911F06C02AE0B701A601CE010E94932A9E
:10560000CDB7DEB7E8E00C94422E9A01AB016627D5
:1056100057FD6095762F0E94CF2A08950F931F9310
:10562000CF93DF93EC019A01AB01662757FD60959C
:10563000762F0E94CF2A8C01CE010E94492A800F2A
:10564000911FDF91CF911F910F9108952115310581
:1056500049F4DC01ED91FC910190F081E02D642F83
:10566000099508950E94932A08959A01462F50E0C3
:1056700060E070E00E94262B08959A01AB0160E083
:1056800070E00E94262B08950F931F93CF93DF9312
:10569000EC010E94262B8C01CE010E94492A800F2A
:1056A000911FDF91CF911F910F9108950F931F9339
:1056B000CF93DF93EC019A01AB0160E070E00E94B0
:1056C000262B8C01CE010E94492A800F911FDF9169
:1056D000CF911F910F9108950F931F93CF93DF9355
:1056E000EC019A01462F50E060E070E00E94262B0A
:1056F0008C01CE010E94492A800F911FDF91CF912A
:105700001F910F910895FC0124853585F901E05C16
:10571000FF4F80819181F901EE5BFF4F2081318144
:10572000821B930B8F7399270895FC0184859585BF
:10573000FC01E05CFF4F40815181FC01EE5BFF4FBB
:10574000208131814217530741F00190F081E02D13
:10575000E80FF91F808190E008958FEF9FEF089583
:10576000FC0184859585FC01E05CFF4F40815181FF
:10577000FC01EE5BFF4F208131814217530779F026
:10578000A081B181A80FB91F8C91208131812F5F39
:105790003F4F2F7333273183208390E008958FEF9D
:1057A0009FEF0895FC0181A1882329F0A489B58980
:1057B0008C9186FFFBCF11A20895CF93DF93FC015C
:1057C00026853785D901A05CBF4F8D919C9111979B
:1057D00001968F739927E901CE5BDF4F488159818C
:1057E00084179507D9F30D90BC91A02DA20FB31F7C
:1057F0006C93A685B785A05CBF4F11969C938E9342
:10580000A689B7892C9181E090E0078C02C0880FAF
:10581000991F0A94E2F7282B2C9381E081A3048836
:10582000F589E02D80818064808381E090E0DF91C4
:10583000CF91089508951F920F920FB60F921124E1
:105840002F933F934F938F939F93EF93FF93809169
:10585000C00082FD1CC04091C600809188069091D6
:10586000890601968F73992720918A0630918B06BD
:105870008217930771F0E0918806F0918906E85B42
:10588000F94F4083909389068093880602C08091E7
:10589000C600FF91EF919F918F914F913F912F9172
:1058A0000F900FBE0F901F90189582EE95E00E940A
:1058B000832B892B11F00E941A2C08951F920F92AE
:1058C0000FB60F9211242F933F938F939F93EF93D3
:1058D000FF932091440630914506809146069091B1
:1058E00047062817390731F48091C1008F7D8093D6
:1058F000C10014C0E0914606F0914706EC5FF94FF5
:105900002081809146069091470601968F739927D2
:1059100090934706809346062093C600FF91EF912F
:105920009F918F913F912F910F900FBE0F901F90DD
:105930001895A0E0B0E0EFE9FCE20C94222EFC0107
:105940001382128288EE93E0A0E0B0E08483958316
:10595000A683B7838CEB93E09183808375876487FC
:1059600057874687318B208B138B028BF58AE48A0D
:10597000D78AC68AB18EA08E938E828E8F85848FB1
:105980008889858F8989868F8A89878F8B8980A36B
:10599000ECE00C943E2ECF92DF92EF92FF92CF93E9
:1059A000DF93EC016A017B01411581EE5807610527
:1059B0007105F9F0EC89FD8981E090E008A002C052
:1059C000880F991F0A94E2F7808360E079E08DE305
:1059D00090E0A70196010E94DB2D21503109410979
:1059E00051095695479537952795211580E1380738
:1059F00098F0EC89FD89108260E874E88EE190E00F
:105A0000A70196010E94DB2D21503109410951095E
:105A10005695479537952795E889F9893083EA891E
:105A2000FB89208319A2EE89FF89408181E090E003
:105A30009C010C8C02C0220F331F0A94E2F7422B08
:105A40004083EE89FF8940819C010D8C02C0220FAA
:105A5000331F0A94E2F7422B4083EE89FF8940818D
:105A60009C010E8C02C0220F331F0A94E2F7422BD6
:105A70004083EE89FF8920810F8C02C0880F991F17
:105A80000A94E2F7809582238083DF91CF91FF9083
:105A9000EF90DF90CF9008958F929F92AF92BF9238
:105AA000CF92DF92EF92FF920F931F9381E08F933B
:105AB00085E08F9387E08F9383E08F9384E08F93CB
:105AC000E6EC8E2E912CF2ECAF2EB12CA1ECCA2E6E
:105AD000D12CB0ECEB2EF12C04EC10E025EC30E0F6
:105AE00044E056E068E476E082EE95E00E94992C6E
:105AF0000F900F900F900F900F901F910F91FF90AC
:105B0000EF90DF90CF90BF90AF909F908F900895CF
:105B10000E94CC280E943322C5E5DCE20E94D124F9
:105B20002097E1F30E94552CF9CFA29FB001B39FBB
:105B3000C001A39F700D811D1124911DB29F700D96
:105B4000811D1124911D08950E94952DA59F900DF2
:105B5000B49F900DA49F800D911D11240895B7FF4F
:105B60000C94A42D0E94A42D821B930B0895DB019D
:105B70008F939F930E94A42DBF91AF91A29F800D00
:105B8000911DA39F900DB29F900D1124089597FB36
:105B9000072E16F4009407D077FD09D00E94592EE5
:105BA00007FC05D03EF4909581959F4F0895709520
:105BB00061957F4F0895A1E21A2EAA1BBB1BFD0120
:105BC0000DC0AA1FBB1FEE1FFF1FA217B307E407DC
:105BD000F50720F0A21BB30BE40BF50B661F771F34
:105BE000881F991F1A9469F7609570958095909514
:105BF0009B01AC01BD01CF010895052E97FB1EF45A
:105C000000940E94142E57FD07D00E94DB2D07FC44
:105C100003D04EF40C94142E509540953095219558
:105C20003F4F4F4F5F4F08959095809570956195C8
:105C30007F4F8F4F9F4F08952F923F924F925F92C9
:105C40006F927F928F929F92AF92BF92CF92DF928C
:105C5000EF92FF920F931F93CF93DF93CDB7DEB7F1
:105C6000CA1BDB0B0FB6F894DEBF0FBECDBF099485
:105C70002A88398848885F846E847D848C849B84DC
:105C8000AA84B984C884DF80EE80FD800C811B81EA
:105C9000AA81B981CE0FD11D0FB6F894DEBF0FBE19
:105CA000CDBFED010895EE0FFF1F0590F491E02D9B
:105CB0000994AA1BBB1B51E107C0AA1FBB1FA61753
:105CC000B70710F0A61BB70B881F991F5A95A9F7A5
:105CD00080959095BC01CD0108958F929F92AF92CF
:105CE000BF92CF92DF92EF92FF92CF93DF93EC01BE
:105CF000688179818A819B81611571058105910592
:105D000021F464E279ED8BE597E02DE133EF41E09A
:105D100050E00E94FD2D49015A019B01AC01A7EA08
:105D2000B1E40E94A42D6B017C01ACEEB4EFA5019F
:105D300094010E94B22DC60ED71EE81EF91EF7FE72
:105D400006C081E0C81AD108E10880E8F80AC882D4
:105D5000D982EA82FB82C701B6019F77DF91CF919A
:105D6000FF90EF90DF90CF90BF90AF909F908F907B
:105D700008950E946D2E089586E091E00E946D2E98
:105D80000895609306017093070180930801909332
:105D9000090108952F923F925F926F927F928F92A6
:105DA0009F92AF92BF92CF92DF92EF92FF920F93AA
:105DB0001F93CF93DF938B01EA016115710521F0E9
:105DC000DB018C9311969C93209739F09E01225011
:105DD00031092332310508F0D8C07C016701BFEFDB
:105DE000CB1ADB0A5601F7016080862D90E00E94F5
:105DF000FC2F892B11F07601F1CFFDE26F120AC062
:105E0000570182E0A80EB11CD70111966C9077243F
:105E100073940BC0BBE26B1207C05701E2E0AE0EF9
:105E2000B11CD70111966C90712CCE018F7E892BFD
:105E300089F4B0E36B1237C0F50180818F7D88351E
:105E4000D1F46180F2E0AF0EB11C872D8260782E14
:105E5000C0E1D0E0CA30D10551F1C031D10521F007
:105E6000C830D10599F409C0CC24CA94DC2CEC2CA0
:105E7000AFE0FA2E22C0209769F7C8E0D0E0CC242A
:105E8000CA94DC2CEC2CFFE1FF2E17C06FEF7FEFE4
:105E9000CB019E01442737FD4095542F0E94DB2DF6
:105EA00069017A010AC02097A9F6CAE0D0E0E9E9C1
:105EB000CE2EDC2CEC2CE9E1FE2EF50160E020E09A
:105EC00030E0A9014E01AA2497FCA094BA2C1F012E
:105ED00070ED572E560CA9E0A51570F48FEB860DCA
:105EE0008A3118F499EC592E06C08FE9860D8A3153
:105EF00048F589EA582E560C852D90E08C179D07A1
:105F00000CF56F3FD9F0C216D306E406F50698F0FB
:105F1000C501B4010E94B72D9B01AC01852D90E015
:105F2000A0E0B0E0280F391F4A1F5B1F2817390770
:105F30004A075B0710F46FEF01C061E03196D101B1
:105F40006C90C5CF0115110551F0662311F0319702
:105F500003C071FE04C03297D801ED93FC9370FE2C
:105F600007C050954095309521953F4F4F4F5F4F5B
:105F700067FF10C082E290E090938D0680938C06BC
:105F80006FEF7FEF8FEF9FEF07C060E070E080E082
:105F900090E002C0B901CA01DF91CF911F910F912A
:105FA000FF90EF90DF90CF90BF90AF909F908F9039
:105FB0007F906F905F903F902F900895FC0188270D
:105FC0009927E89421912032E9F3293010F02E30FE
:105FD000C8F32B3241F02D3239F4689404C00E948A
:105FE0003030820F911D219120532A30C0F31EF4CE
:105FF000909581959F4F0895911150C0803219F06E
:1060000089508550D0F7089548EC53E00E9409303C
:106010000895FA01A191B081009719F41097E1F069
:10602000CD01DC01CD010D90002011F4C00113C0A1
:10603000FB012191222319F02015D9F7F3CFFB01A1
:106040002191201519F41E92119606C02223C1F742
:106050000D900020A1F7D001FA01A193B08308951B
:106060007AE0979F902D879F802D910D11240895A0
:10607000F999FECF92BD81BDF89A992780B5089510
:10608000262FF999FECF1FBA92BD81BD20BD0FB654
:10609000F894FA9AF99A0FBE0196089599278827DD
:0660A0000895F894FFCF03
:1060A60000008E06200001000000FF000200020032
:1060B60002000200020002000200020002000200CA
:1060C6000200020002000200020002802500000514
:1060D600400AA1204EA50020244EA52C2330C01234
:1060E60000001A400AA1204EA5001B1E27522C2391
:1060F600308025000005400AA1204EA50020244E30
:10610600A52C2330004B000006400AD0009D490014
:106116007B289D492C233000E1000005400A4501FB
:10612600D7DC03B81E0EBF00232E48E801008A40C4
:106136000A6001555502AD1E20000023C8015458BF
:106146002074696D656F75742100596573004E6F13
:10615600002C00386368004E2F41002C205B005D48
:106166002028002900486F70206368616E6E656C98
:10617600200020402000456E746572696E672061BC
:1061860064617074697665206368616E6E656C2003
:1061960073656C656374696F6E2C207069636B69D7
:1061A6006E673A007363616E6E6572206D6F64652B
:1061B600004E4F5420454E41424C45440053656EB7
:1061C60064696E672073657474696E677320746F93
:1061D6002052580A00526573657474696E6720739D
:1061E600657474696E6773206F6E2052580A004199
:1061F600626F727465642065646974730A00696EFF
:1062060076616C69642073656C656374696F6E0092
:106216000D0A496E76616C696420696E707574202A
:106226002D20646973636172646564210700536598
:106236007474696E677320736176656420746F2069
:10624600454550524F4D0A00526576657274656435
:106256002073657474696E67732066726F6D20456E
:106266004550524F4D0A004C6F616465642066616B
:1062760063746F72792064656661756C74730A0065
:106286004B657920616E64206368616E6E656C7320
:106296002072616E646F6D697A65640A004F70657D
:1062A6006E4C52536E672054582073746172746931
:1062B6006E672000206F6E20485720006D6F647552
:1062C6006C65206C6F636B65643F00342B3400385B
:1062D60000382B340031320031322B340031360095
:1062E60050504D0052535349005344410053434CC0
:1062F60000525844005458440041494E004C42450F
:1063060045500053504B54524D0053425553005381
:10631600554D44004C4C494E440000070B0C1011DF
:106326001500B7012B032F033103350338033D0353
:10633600B7014003440349034D0351035503590371
:106346005D0363036A036F0374038D028D028D027E
:106356008D02160A1322312900000000DD2BE229E6
:08636600832BB02B952BD22BE9
:107E00000F92CDB7DEB7112484B714BE81FFF1D035
:107E100082E08093C00088E18093C10086E0809377
:107E2000C20080E18093C4008EE0CDD088249924E4
:107E3000CC24C394F5E0DF2EE1E1EE2E73E0F72EC3
:107E4000B6D0082F813479F4B2D08983C2D0898129
:107E5000823811F481E005C0813811F485E001C059
:107E600083E09ED09AC0823411F484E103C085344B
:107E700019F485E0B6D091C0853561F498D0082F0B
:107E800010E095D090E0982E8824802A912A880CC2
:107E9000991C82C0863521F484E0A3D080E0E1CF34
:107EA000843609F04CC083D082D0A82E80D0B82E62
:107EB00000E011E07CD0F80181938F01AE16D1F77C
:107EC00088D0FB2DF53489F4E0E0F1E00BC0F9999E
:107ED000FECF92BC81BC0894811C911C819180BD15
:107EE000FA9AF99AEA1598F358C08B2D863409F05E
:107EF00054C0F401F7BEE89507B600FCFDCFF401CD
:107F0000A0E0B1E02C9130E011968C91119790E0B7
:107F1000982F8827822B932B12960C01C7BEE895C9
:107F20001124329681E0A038B80761F7F401D7BE7A
:107F3000E89507B600FCFDCFE7BEE8952EC0843774
:107F4000F1F435D034D0182F32D0B82E42D0FB2DDA
:107F5000F63421F4F40105914F010CC0FB2DF534EA
:107F600049F4F999FECF92BC81BC0894811C911C04
:107F7000F89A00B5802F14D0115049F70EC08537FC
:107F800039F427D08EE10CD085E90AD08FE069CF93
:107F9000813511F488E017D01CD080E101D050CF9A
:107FA0009091C00095FFFCCF8093C600089580910A
:107FB000C00087FFFCCF8091C00084FD01C0A89560
:107FC0008091C6000895E0E6F0E098E19083808318
:107FD0000895EDDF803219F088E0F5DFFFCF84E10E
:107FE000DFCF1F93182FE3DF1150E9F7F2DF1F9166
:0E7FF0000895282E80E0E7DFEE27FF27099492
:027FFE0001057B
:0400000300007E007B
:00000001FF
